:101CD000AF61EFC4135407FFEF30E032E516701622
:101CE000E5177012E518700EAF60EF54EFF560AFB6
:101CF00060EF54F7F560E51D6005E51DB480087FD1
:0F1D0000017E00120BCF227F007E00120BCF223C
:040BCF008E428F4380
:100BD300E54345427003020CC7AF23EFC41313541C
:100BE30003FFEF20E020AF22EF131313541FFFEF97
:100BF30020E013AF5FEFC413135403FFEF20E006AD
:100C0300AF23EF30E0D3C2AFAF23EF54BFF523D20E
:100C1300AF90702C7404F0AE26AF27E4FCFDAB2D2F
:100C2300AA2CA92BA82AD312154E40088526448541
:100C330027458008AE2CAF2D8E448F45AF61EF3032
:100C4300E028756200756300C3E5639545E5629529
:100C530044503D907020E0FFAE6374642EF8A60705
:100C63000563E5637002056280DE756200756300EB
:100C7300C3E5639545E56295445015907020E0FF08
:100C83007E008E5C8F5D0563E5637002056280E024
:100C9300AE44AF45AB07AA06E4F9F8C3E52D9BF5CF
:100CA3002DE52C9AF52CE52B99F52BE52A98F52AB9
:100CB300AF2DAE2CAD2BAC2AEC4D4E4F6003020B87
:100CC300DC020DDE90702C7405F0AE26AF27E4FC39
:100CD300FDAB2DAA2CA92BA82AD312154E4019AF70
:100CE3002790701CEFF0E526FF7E0090701DEFF05B
:100CF3008526448527458021AF2D90701CEFF0AFEA
:100D03002DAE2CAD2BAC2A780812155F90701DEF19
:100D1300F0AE2CAF2D8E448F45AF61EF30E02875D8
:100D23006200756300C3E5639545E5629544503BF6
:100D3300AF6374642FF8E6FF907020EFF00563E56E
:100D4300637002056280DE756200756300C3E5634C
:100D53009545E562954450137E00AF63907020EF94
:100D6300F00563E5637002056280E2AF23EFC4130D
:100D730013135401FFEF20E020AF22EF131313549A
:100D83001FFFEF20E013AF5FEFC413135403FFEF14
:100D930020E006AF23EF30E0D2C2AFAF23EF547FA2
:100DA300F523D2AFAE44AF45AB07AA06E4F9F8C3C7
:100DB300E52D9BF52DE52C9AF52CE52B99F52BE5E7
:100DC3002A98F52AAF2DAE2CAD2BAC2AEC4D4E4F05
:100DD3006003020CC7756200756300AF61EF54DFF7
:020DE300F561B8
:010DE50022EB
:04000600024F700035
:1015F500758E02758F01D292752D00752C00752B95
:1016050000752A00752600752740754E00AF14EF4A
:101615005400FFEF4404F514121D92C29290700C11
:10162500E0FFEF54FEFF90700CEFF0C2B47F647ED4
:1016350000121A92D2B47F647E00121A92AE4FAF96
:10164500508F828E83E5822471F582E5833400F51F
:1016550083E0FFEFB481D4AE4FAF508F828E83E528
:10166500822472F582E5833400F583E0FFEFB4153B
:10167500BA75250075240075230075220075530081
:10168500755400756100756000755F00755E00AF8B
:0C16950061EF4401F561D290121D6A2241
:101D9200758901754A07754BD0754C4E754D207586
:101DA2008800C2AF75A80275B800D2BBD2B9D2AF53
:041DB20075874022CF
:101D6A00121DD7120916AF12EF541FF5127555003E
:101D7A00AF15EF54FEF515AF15EF4440F515AF60FA
:081D8A00EF54DFF560D2A8223E
:101DD70090700CE0FFEF448CFF90700CEFF0907068
:0F1DE700107454F090701412159139FD00002201
:10091600AF61EF20E003020A6F90702C7402F09032
:1009260070047440F0A3E4F090702C7403F090709F
:10093600047440F0A3E4F090702C7404F0907004FA
:100946007440F0A3E4F090702C7405F09070047479
:1009560040F0A3E4F090702C7406F090700474409C
:10096600F0A3E4F090702C7407F09070047440F0DB
:10097600A3E4F090702C7402F09070087417F0A342
:10098600E4F090702C7403F09070087417F0A3E4F0
:10099600F090702C7404F09070087416F0A3E4F0D4
:1009A60090702C7405F09070087416F0A3E4F09023
:1009B600702C7406F09070087415F0A3E4F0907033
:1009C6002C7407F09070087415F0A3E4F090702C66
:1009D6007402F0907008E0FEA3E0FFEE4408FE907B
:1009E6007008EEF0A3EFF090702C7403F09070088E
:1009F600E0FEA3E0FFEE4408FE907008EEF0A3EFE1
:100A0600F090702C7404F0907008E0FEA3E0FFEE06
:100A16004408FE907008EEF0A3EFF090702C740579
:100A2600F0907008E0FEA3E0FFEE4408FE90700828
:100A3600EEF0A3EFF090702C7406F0907008E0FED4
:100A4600A3E0FFEE4408FE907008EEF0A3EFF090EE
:100A5600702C7407F0907008E0FEA3E0FFEE4408E7
:100A6600FE907008EEF0A3EFF0AF61EF30E0030206
:100A76000BC890702C7402F09070047440F0A3E4DC
:100A8600F090702C7403F09070047440F0A3E4F0BE
:100A960090702C7404F0907004E4F0A37402F0904B
:100AA600702C7405F0907004E4F0A37402F090705A
:100AB6002C7406F09070047440F0A3E4F090702C4F
:100AC6007407F09070047440F0A3E4F090702C74F6
:100AD60002F09070087417F0A3E4F090702C740381
:100AE600F09070087417F0A3E4F090702C7404F082
:100AF6009070087416F0A3E4F090702C7405F090D2
:100B060070087416F0A3E4F090702C7406F09070E0
:100B1600087415F0A3E4F090702C7407F090700838
:100B26007415F0A3E4F090702C7402F0907008E055
:100B3600FEA3E0FFEE4408FE907008EEF0A3EFF08F
:100B460090702C7403F0907008E0FEA3E0FFEE4472
:100B560008FE907008EEF0A3EFF090702C7404F08D
:100B6600907008E0FEA3E0FFEE4408FE907008EEE9
:100B7600F0A3EFF090702C7405F0907008E0FEA3DF
:100B8600E0FFEE4408FE907008EEF0A3EFF09070E0
:100B96002C7406F0907008E0FEA3E0FFEE4408FE19
:100BA600907008EEF0A3EFF090702C7407F0907040
:100BB60008E0FEA3E0FFEE4408FE907008EEF0A306
:090BC600EFF09070007480F02241
:0300130002000EDA
:01000E0032BF
:03001B0002000FD1
:01000F0032BE
:03002300020010C8
:0100100032BD
:03002B00020011BF
:0100110032BC
:03000B00021E25AD
:101E2500C0E0C0D075D000AF5FEF4420F55FD0D0E3
:031E3500D0E032C8
:030003000219A03F
:1019A000C0E0C0F0C083C082C0D075D0089070186D
:1019B000E0FCA3E0FDA3E0FEA3E0FFE5254FF52555
:1019C000E5244EF524E5234DF523E5224CF522AF21
:1019D00025AE24AD23AC22907018121585AF22EFEE
:1019E00030E02EAF22EF54FEF522AF5FEF4440F51A
:1019F0005F752600752740D290AF61EF4401F56115
:101A0000121D6A90700CE0FFEF4401FF90700CEF24
:0C1A1000F0D0D0D082D083D0F0D0E032F3
:101BC1001215F590700CE0FFEF4401FF90700CEFDF
:101BD100F01216A1121CD0AF23EFC4540FFFEF3047
:101BE100E026AF23EF54EFF5237B007A0079327DB5
:101BF100087C007F02121A1C8E308F3175320075FD
:101C010033127534127535127B007A0079327D04F6
:0D1C11007C007F03121AFA8E308F3180B4F0
:011C1E0022A3
:101A92008E428F43854A5C854B5DC374FF955DF52D
:101AA2005D74FF955CF55CD2A9E55CF55D755C0043
:101AB200855D8C854A5C854B5DC374FF955DF55DE4
:101AC20074FF955CF55C855D8AD28CAF5FEF54DF65
:101AD200F55FAF5FEFC4135407FFEF30E0F4AF5F81
:101AE200EF54DFF55FC28CC2A9E5431543700215BE
:081AF20042E5434542709D22CC
:101293001201100100000040CC04491B00000102B0
:1012A30000011201000200000040CC04491B0000B1
:1012B300010200010A0600020000004001000902C9
:1012C3002E00010100C03209072E00010100C032C7
:1012D30009040000040000000009040000040000E9
:1012E30000000705020240000007058202400000DB
:1012F300070502020002000705820200020007053B
:1013030001034000010705810340000107050103B4
:1013130040000107058103400001090400010200A8
:101323000000000705030140000107058301400099
:1013330001070503010000010705830100000130D7
:10134300035000680069006C00690070007300209E
:1013530000490053005000310035003800310020AF
:1013630000560065007200200031002E003000009E
:101373000000000000000000000000000000001C4E
:10138300035000680069006C006900700020002DA4
:101393000020004100500049004300000000000409
:1013A300030904C3000000000000000000AAAAAA69
:1013B300AAAAAAAAAAEEEEEEEEEEEEEEEEFEFFFF6C
:1013C300FFFFFFFFFFFFFFFFFF7FBFDFEFF7FBFD28
:0B13D300FC7EBFDFEFF7FBFD7EB6CE17
:101D0F00FF17E3FF0DE6FF0012FF0F94FF0012FF16
:101D1F001D3FFF002EFF0012FF1DB6FF1744FF18D7
:101D2F007EFF1B5EFF0012FF0012FF0012FF00126A
:1016A100AF23EF30E007C2AF121134D2AFAF22EF58
:1016B100131313541FFFEF30E027C2AFAF22EF54D3
:1016C100F7F522D2AF90700CE0FFEF4420FF90704D
:1016D1000CEFF090700CE0FFEF54DFFF90700CEF17
:1016E100F0AF22EFC4540FFFEF30E027C2AFAF22BB
:1016F100EF54EFF522D2AF90700CE0FFEF4440FFC2
:1017010090700CEFF090700CE0FFEF54BFFF907001
:101711000CEFF0AF22EFC4135407FFEF30E023C208
:10172100AFAF22EF54DFF522D2AFAF61EF30E0125D
:10173100C290AF61EF54FEF561120916752602756C
:031741002700225C
:10113400AF23EF54FEF523AF5FEF54BFF55F90701C
:101144002C7420F0907020E0FF78A4A60790702003
:10115400E0FF78A5A607907020E0FF7E0078A6A6A1
:101164000608A60778A6E6FE08E6FFEF7F00FE78ED
:10117400A6A60608A60778A6E6FE08E6FF90702055
:10118400E0FD7C00EE4CFEEF4DFF78A6A60608A617
:1011940007907020E0FF7E0078A8A60608A60778CE
:1011A400A8E6FE08E6FFEF7F00FE78A8A60608A6DC
:1011B4000778A8E6FE08E6FF907020E0FD7C00EECC
:1011C4004CFEEF4DFF78A8A60608A607907020E015
:1011D400FF7E0078AAA60608A60778AAE6FE08E617
:1011E400FFEF7F00FE78AAA60608A60778AAE6FE07
:1011F40008E6FF907020E0FD7C00EE4CFEEF4DFF12
:1012040078AAA60608A60778AAE6F55C08E6F55DBE
:1012140078AA7600087600AF5D7E0078AAA6060854
:10122400A60778AAE6FE08E6FFEF7F00FE78AAA6E6
:101234000608A607E55CF55D755C0078AAE6FE087D
:10124400E6FFEE455CFEEF455DFF78AAA60608A61C
:101254000778A4E6FFEF5460F54278A5E6FFEF5463
:101264000FF543E542B440041213DE22E542701E3A
:10127400AF43EF75F003A4240FF582E4341DF58326
:0E128400E493FB740193FA740293F91215EFD0
:011292002239
:1013DE0078A5E6FFEF640C600302152278A8E6FEFE
:1013EE0008E6FFEF8EF01215C2142E71041403726C
:1013FE0004000014A978AAE6FE08E6FFEF64014E89
:10140E00701E90702C7401F090701C7401F090702E
:10141E001DE4F09070207422F0121C1F121E0E227A
:10142E00121C7890702CE4F0907020E0FF8F1690D4
:10143E007020E0FF8F17907020E0FF8F18907020C3
:10144E00E0FF7E008E5C8F5D907020E0FFE4FCFD7F
:10145E00FE8F2D8E2C8D2B8C2AAF2DAE2CAD2BAC62
:10146E002A78081215728F2D8E2C8D2B8C2AAE5C3D
:10147E00AF5DE4FCFDE52D4FF52DE52C4EF52CE58D
:10148E002B4DF52BE52A4CF52A907020E0FF8F1D91
:10149E00121DF6AF61EF4420F5612278A4E6FFEF4E
:1014AE00B4C004121DF62278A4E6FFEF6440706407
:1014BE0090702CE4F0907028E0FFEF4401FF9070E4
:1014CE0028EFF0AF23EF20E044907018E0FCA3E08B
:1014DE00FDA3E0FEA3E0FFE5254FF525E5244EF53F
:1014EE0024E5234DF523E5224CF522AF25AE24ADA0
:1014FE0023AC22907018121585AF22EF13131354DC
:10150E001FFFEF20E00EAF22EF30E0B722AF23EF48
:05151E0054F7F5232243
:0100120022CB
:10002E0078A6E6FE08E6FFEF8EF01215C2005F001E
:10003E000100CC00020359000303CC000403D000DE
:10004E0005060B0006068E000709150008000008BD
:10005E00B0AF61EF30E0087E127F938E1E8F1FAF20
:10006E0061EF20E0087E127FA58E1E8F1FAE1EAFA1
:10007E001F8F828E83E493FF7E008E518F5290707D
:10008E002C7401F090701C7412F090701DE4F0E569
:10009E005245516022AE1EAF1F8F828E83E493FFB6
:1000AE00907020EFF0E552155270021551051FE5C4
:1000BE001F7002051E80D8121C1F121E0E22AF23A7
:1000CE00EF54FBF523755C00755D407E127FC18E8B
:1000DE001E8F1FAE1EAF1F8F828E83E493FF7E0096
:1000EE008E518F5290702C7401F078AAE6FE08E6BD
:1000FE00FFC3E5529FE5519E405878ABE6FF9070E6
:10010E001CEFF078AAE6FE08E6FFEEFF7E00907088
:10011E001DEFF075510075520078AAE6FE08E6FF55
:10012E00C3E5529FE5519E5022AE1EAF1F8F828EA9
:10013E0083E493FF907020EFF0051FE51F7002051A
:10014E001E0552E5527002055180CE121C1F121E62
:10015E000E2278AAE6FE08E6FFC3EF9420EE940086
:10016E005003020344E55245516022AE1EAF1F8F6D
:10017E00828E83E493FF907020EFF0E5521552705B
:10018E00021551051FE51F7002051E80D8AF61EFE5
:10019E0030E0087E127FD38E1E8F1FAF61EF20E0FE
:1001AE00087E127FDC8E1E8F1FAE1EAF1F8F828EBB
:1001BE0083E493FF7E008E518F52E55245516022AB
:1001CE00AE1EAF1F8F828E83E493FF907020EFF0F0
:1001DE00E552155270021551051FE51F7002051EDE
:1001EE0080D8AF61EF30E0087E137F088E1E8F1F20
:1001FE00AF61EF20E0087E137F168E1E8F1FAE1E9E
:10020E00AF1F8F828E83E493FF7E008E518F52E557
:10021E005245516022AE1EAF1F8F828E83E493FF34
:10022E00907020EFF0E552155270021551051FE542
:10023E001F7002051E80D8AF61EF30E0087E137F7D
:10024E00018E1E8F1FAF61EF20E0087E137F0F8E91
:10025E001E8F1FAE1EAF1F8F828E83E493FF7E0014
:10026E008E518F52E55245516022AE1EAF1F8F82C6
:10027E008E83E493FF907020EFF0E55215527002DA
:10028E001551051FE51F7002051E80D8AF61EF30B6
:10029E00E0087E127FEC8E1E8F1FAF61EF20E0080C
:1002AE007E127FFA8E1E8F1FAE1EAF1F8F828E8321
:1002BE00E493FF7E008E518F52E55245516022AE7F
:1002CE001EAF1F8F828E83E493FF907020EFF0E5B8
:1002DE0052155270021551051FE51F7002051E8042
:1002EE00D8AF61EF30E0087E127FE58E1E8F1FAF14
:1002FE0061EF20E0087E127FF38E1E8F1FAE1EAFC1
:10030E001F8F828E83E493FF7E008E518F52E552B3
:10031E0045516022AE1EAF1F8F828E83E493FF90F5
:10032E007020EFF0E552155270021551051FE51FB2
:10033E007002051E80D8907028E0FFEF4408FF90F1
:10034E007028EFF0121C1F121E0E227E137FA28E3B
:10035E001E8F1FAE1EAF1F8F828E83E493FF7E0013
:10036E008E518F5290702C7401F078AAE6FE08E63A
:10037E00FFC3EF9552EE9551500978AAE6F5510854
:10038E00E6F552AF5290701CEFF090701DE4F0E560
:10039E005245516022AE1EAF1F8F828E83E493FFB3
:1003AE00907020EFF0051FE51F7002051EE5521537
:1003BE00527002155180D8121C1F121E0E221200EE
:1003CE001222755C00755D0078A6E6FE08E6FF7EDB
:1003DE0000D3EF9401EE94004063907028E0FFEF9D
:1003EE004401FF907028EFF0AF23EF20E0479070AC
:1003FE0018E0FCA3E0FDA3E0FEA3E0FFE5254FF52A
:10040E0025E5244EF524E5234DF523E5224CF52272
:10041E00AF25AE24AD23AC22907018121585AF22F5
:10042E00EF131313541FFFEF30E003020915AF2231
:10043E00EF30E0B422AF23EF54F7F523227E127F84
:10044E00E58E1E8F1FAE1EAF1F8F828E83E493FF2D
:10045E007E008E518F5290702C7401F078AAE6FEB9
:10046E0008E6FFC3E5529FE5519E405978AAE6F58E
:10047E005C08E6F55DAF5D90701CEFF0E55CFF7E0D
:10048E000090701DEFF075510075520078AAE6FECF
:10049E0008E6FFC3E5529FE5519E5022AE1EAF1FE8
:1004AE008F828E83E493FF907020EFF0051FE51F7F
:1004BE007002051E0552E5527002055180CE121CC7
:1004CE001F121E0E2278AAE6FE08E6FFC3EF955213
:1004DE00FFEE9551FE78AAA60608A607E552255D01
:1004EE00F55DE551355CF55CE55245516022AE1E79
:1004FE00AF1F8F828E83E493FF907020EFF0E55252
:10050E00155270021551051FE51F7002051E80D889
:10051E007E127FEC8E1E8F1FAE1EAF1F8F828E83BC
:10052E00E493FF7E008E518F5278AAE6FE08E6FF16
:10053E00C3E5529FE5519E406178AAE6FE08E6FFAC
:10054E00EF255DF55DEE355CF55CAF5D90701CEFF3
:10055E00F0E55CFF7E0090701DEFF0755100755256
:10056E000078AAE6FE08E6FFC3E5529FE5519E50CD
:10057E0022AE1EAF1F8F828E83E493FF907020EF0A
:10058E00F0051FE51F7002051E0552E552700205AB
:10059E005180CE121C1F121E0E2278AAE6FE08E60D
:1005AE00FFC3EF9552FFEE9551FE78AAA60608A658
:1005BE0007E552255DF55DE551355CF55CAF5D9067
:1005CE00701CEFF0E55CFF7E0090701DEFF0E552C1
:1005DE0045516022AE1EAF1F8F828E83E493FF9033
:1005EE007020EFF0E552155270021551051FE51FF0
:1005FE007002051E80D8121C1F121E0E227E127F44
:10060E00B78E1E8F1FAE1EAF1F8F828E83E493FF99
:10061E007E008E518F5290702C7401F078AAE6FEF7
:10062E0008E6FFC3EF9552EE9551501978ABE6FFF1
:10063E0090701CEFF090701DE4F078AAE6F551086A
:10064E00E6F552800CAF5290701CEFF090701DE4E6
:10065E00F0E55245516022AE1EAF1F8F828E83E4AD
:10066E0093FF907020EFF0051FE51F7002051EE549
:10067E005215527002155180D8121C1F121E0E22D6
:10068E00755C00755D407E127FCA8E1E8F1FAE1E7A
:10069E00AF1F8F828E83E493FF7E008E518F529018
:1006AE00702C7401F078AAE6FE08E6FFC3E5529FAF
:1006BE00E5519E405878ABE6FF90701CEFF078AA9B
:1006CE00E6FE08E6FFEEFF7E0090701DEFF075511E
:1006DE000075520078AAE6FE08E6FFC3E5529FE5D4
:1006EE00519E5022AE1EAF1F8F828E83E493FF90D9
:1006FE007020EFF0051FE51F7002051E0552E55232
:10070E007002055180CE121C1F121E0E2278AAE610
:10071E00FE08E6FFC3EF9420EE9400500302089B00
:10072E00E55245516022AE1EAF1F8F828E83E49339
:10073E00FF907020EFF0E552155270021551051F13
:10074E00E51F7002051E80D87E127FD38E1E8F1F6E
:10075E00AE1EAF1F8F828E83E493FF7E008E518F6D
:10076E0052E55245516022AE1EAF1F8F828E83E43A
:10077E0093FF907020EFF0E552155270021551055F
:10078E001FE51F7002051E80D87E137F088E1E8FF8
:10079E001FAE1EAF1F8F828E83E493FF7E008E519D
:1007AE008F52E55245516022AE1EAF1F8F828E834F
:1007BE00E493FF907020EFF0E55215527002155140
:1007CE00051FE51F7002051E80D87E137F018E1E49
:1007DE008F1FAE1EAF1F8F828E83E493FF7E008E1F
:1007EE00518F52E55245516022AE1EAF1F8F828E41
:1007FE0083E493FF907020EFF0E5521552700215CE
:10080E0051051FE51F7002051E80D87E127FEC8EEB
:10081E001E8F1FAE1EAF1F8F828E83E493FF7E004E
:10082E008E518F52E55245516022AE1EAF1F8F8200
:10083E008E83E493FF907020EFF0E5521552700214
:10084E001551051FE51F7002051E80D87E127FE52B
:10085E008E1E8F1FAE1EAF1F8F828E83E493FF7E80
:10086E00008E518F52E55245516022AE1EAF1F8F42
:10087E00828E83E493FF907020EFF0E55215527054
:10088E00021551051FE51F7002051E80D8907028B5
:10089E00E0FFEF4408FF907028EFF0121C1F121EAD
:1008AE000E2290702C7401F0907028E0FFEF44013E
:1008BE00FF907028EFF0AF23EF20E044907018E027
:1008CE00FCA3E0FDA3E0FEA3E0FFE5254FF525E543
:1008DE00244EF524E5234DF523E5224CF522AF25D4
:1008EE00AE24AD23AC22907018121585AF22EF13F3
:1008FE001313541FFFEF20E00EAF22EF30E0B722AC
:08090E00AF23EF54F7F523229B
:101D3F00AF23EF54FBF52378A6E6FE08E6FFEEFF90
:101D4F007E00EF547FFF907000E0FEEE5480FEEEB9
:0B1D5F004FFF907000EFF0121DF62205
:10174400AF23EF54FBF52378A6E6FE08E6FFEF4E41
:101754007007755500121DF62278A6E6FE08E6FF0E
:10176400EFB40015EEB4011178A6E6FE08E6FFEE2C
:10177400FF7E008F55121DF62290702C7401F0909C
:101784007028E0FFEF4401FF907028EFF0AF23EFE3
:1017940020E044907018E0FCA3E0FDA3E0FEA3E089
:1017A400FFE5254FF525E5244EF524E5234DF523E6
:1017B400E5224CF522AF25AE24AD23AC229070185F
:1017C400121585AF22EF131313541FFFEF20E00E01
:0F17D400AF22EF30E0B722AF23EF54F7F5232217
:101DB60090702C7401F0907020E555F0907028E03A
:101DC600FFEF4408FF907028EFF0121C1F121E0E42
:011DD60022EA
:100DE60078A4E6FFEF540FF544E54464026003027D
:100DF6000F1078A6E6FE08E6FFEF4E6003020F101E
:100E060078A8E6FE08E6FFEF8EF01215C20E5F0028
:100E1600000E6E01000E7E02000E8E03000E9E0472
:100E2600000EAE05000EBE06000ECE07000E578061
:100E3600000E6681000E7682000E8683000E968472
:100E4600000EA685000EB686000EC6870000000EB0
:100E5600D490702C7401F0807590702CE4F0806E44
:100E660090702C7403F0806690702C7402F0805E93
:100E760090702C7405F0805690702C7404F0804E9F
:100E860090702C7407F0804690702C7406F0803EAB
:100E960090702C7409F0803690702C7408F0802EB7
:100EA60090702C740BF0802690702C740AF0801EC3
:100EB60090702C740DF0801690702C740CF0800ECF
:100EC60090702C740FF0800690702C740EF0907059
:100ED60028E0FFEF54FEFF907028EFF0AF60EF546C
:100EE6007FF560907008E0FFEF54F7FF907008EF11
:100EF600F0907008E0FFEF4408FF907008EFF012E2
:100F06001DF6AF12EF54FDF51222E544701A78A6CD
:100F1600E6FE08E6FFEFB4000FEEB4010BAF12EFEA
:100F260054FEF512121DF62290702C7401F090708A
:100F360028E0FFEF4401FF907028EFF0AF23EF2089
:100F4600E044907018E0FCA3E0FDA3E0FEA3E0FF00
:100F5600E5254FF525E5244EF524E5234DF523E556
:100F6600224CF522AF25AE24AD23AC229070181288
:100F76001585AF22EF131313541FFFEF20E00EAFBA
:0D0F860022EF30E0B722AF23EF54F7F52340
:010F9300223B
:1017E30078A4E6FFEFB4802290702C7401F090701F
:1017F3001C7402F090701DE4F09070207401F0905E
:101803007021E4F0121C1F121E0E78A4E6FFEFB441
:10181300812190702C7401F090701C7402F0907010
:101823001DE4F0907020E4F0907021E4F0121C1F8E
:10183300121E0E78A4E6FFEF6482703E755C00759D
:101843005D00AF12EFC313FFEF5401FF7E008E5C08
:101853008F5D90702C7401F090701C7402F0907086
:101863001DE4F0AF5D907020EFF0E55CFF7E00902B
:0B1873007021EFF0121C1F121E0E224D
:100F940078A4E6FFEF540FF544E5446402600302CD
:100FA40010B078A6E6FE08E6FFEF4E60030210B02C
:100FB40078A8E6FE08E6FFEF8EF01215C2100D00C9
:100FC40000101C0100102C0200103C0300104C0403
:100FD40000105C0500106C0600107C0700100580F2
:100FE4000010148100102482001034830010448403
:100FF40000105485001064860010748700000010EF
:101004008290702C7401F0807590702CE4F0806EE6
:1010140090702C7403F0806690702C7402F0805EE3
:1010240090702C7405F0805690702C7404F0804EEF
:1010340090702C7407F0804690702C7406F0803EFB
:1010440090702C7409F0803690702C7408F0802E07
:1010540090702C740BF0802690702C740AF0801E13
:1010640090702C740DF0801690702C740CF0800E1F
:1010740090702C740FF0800690702C740EF09070A9
:1010840028E0FFEF4401FF907028EFF0AF60EF44D9
:1010940080F560907008E0FFEF54F7FF907008EF60
:1010A400F0121DF6AF12EF54FDF51222E544701A4A
:1010B40078A6E6FE08E6FFEFB4000FEEB4010BAF2E
:1010C40012EF4401F512121DF62290702C7401F0F7
:1010D400907028E0FFEF4401FF907028EFF0AF23F9
:1010E400EF20E044907018E0FCA3E0FDA3E0FEA331
:1010F400E0FFE5254FF525E5244EF524E5234DF5E0
:1011040023E5224CF522AF25AE24AD23AC2290700A
:1011140018121585AF22EF131313541FFFEF20E0AD
:0F1124000EAF22EF30E0B722AF23EF54F7F523E1
:011133002299
:10187E0078A6E6FE08E6FFEF4E6060907028E0FF67
:10188E00EF4401FF907028EFF0AF23EF20E044907B
:10189E007018E0FCA3E0FDA3E0FEA3E0FFE5254FFA
:1018AE00F525E5244EF524E5234DF523E5224CF5EB
:1018BE0022AF25AE24AD23AC22907018121585AF41
:1018CE0022EF131313541FFFEF20E039AF22EF3036
:1018DE00E0B722AF23EF54F7F5232290702C74015A
:1018EE00F090701C7401F090701DE4F0AF15EF20B5
:1018FE00E007907020E4F080069070207401F012E2
:06190E001C1F121DF62251
:101B5E0078A8E6FE08E6FFEF4E701678A6E6FE08B9
:101B6E00E6FFEFB4000BEEB40107AF15EF4401F53D
:101B7E001578A8E6FE08E6FFEFB40016EEB40112E3
:101B8E0078A6E6FE08E6FFEF4E7007AF15EF54FE9F
:101B9E00F51578A8E6FE08E6FFEF4E701278A6E679
:101BAE00FE08E6FFEF4E7007AF15EF54FEF5151267
:031BBE001DF622EF
:101DF60090702C7401F0907028E0FFEF4402FF9081
:081E06007028EFF0121C1F22EE
:101C1F00AF23EF131313541FFFEF20E044907018FE
:101C2F00E0FCA3E0FDA3E0FEA3E0FFE5254FF525D3
:101C3F00E5244EF524E5234DF523E5224CF522AF9F
:101C4F0025AE24AD23AC22907018121585AF22EF6C
:101C5F00131313541FFFEF20E00EAF22EF30E0B04D
:091C6F0022AF23EF54F7F5232204
:101E0E0090702CE4F0907028E0FFEF4402FF907089
:071E1E0028EFF0121C7822EE
:101C7800AF23EF1313543FFFEF20E044907018E0B8
:101C8800FCA3E0FDA3E0FEA3E0FFE5254FF525E575
:101C9800244EF524E5234DF523E5224CF522AF2506
:101CA800AE24AD23AC22907018121585AF22EF1325
:101CB8001313541FFFEF20E00EAF22EF30E0B122E4
:081CC800AF23EF54FBF52322CA
:101A1C00D310AF01C3C0D08F428C438D448B458A09
:031A2C00468947A1
:101A2F0090702CE542F090701DE0FF7E008E438F8A
:101A3F0044E544754400F54390701CE0FF7E00EFD1
:101A4F002544F544EE3543F543854348854449E540
:101A5F00491549AE4870021548FFEF4E601C907053
:101A6F0020E0FFAB45AA46A947EF12153C740125AC
:0E1A7F0047F547E43546F54680D5AE43AF4403
:051A8D00D0D092AF2251
:101AFA00D310AF01C3C0D08F428C438D448B458A2B
:031B0A00468947C2
:101B0D0090702CE542F0AF4490701CEFF0E543FF70
:101B1D007E0090701DEFF0854348854449E54915D9
:101B2D0049AE4870021548FFEF4E601CAB45AA4602
:101B3D00A947121523FF907020EFF074012547F58A
:0C1B4D0047E43546F54680D5AE43AF4472
:051B5900D0D092AF2284
:03000000021914CE
:0C191400787FE4F6D8FD7581B102195B04
:10152300BB010689828A83E0225002E722BBFE02C6
:09153300E32289828A83E49322F9
:10153C00BB010689828A83F0225002F722BBFE018E
:02154C00F32288
:10154E00EB9FF5F0EA9E42F0E99D42F0E89C45F0F3
:01155E00226A
:10155F00E8600FECC313FCED13FDEE13FEEF13FF6A
:03156F00D8F1228E
:10157200E8600FEFC333FFEE33FEED33FDEC33FCD7
:03158200D8F1227B
:0C158500ECF0A3EDF0A3EEF0A3EFF022D9
:10159100A8828583F0D083D0821215A81215A812D3
:1015A10015A81215A8E473E493A3C583C5F0C583F8
:1015B100C8C582C8F0A3C583C5F0C583C8C582C8A4
:0115C1002207
:1015C200D083D082F8E4937012740193700DA3A3B8
:1015D20093F8740193F5828883E473740293B5F0EF
:0D15E200067403936860E9A3A3A3A380D857
:0615EF008A838982E47387
:10192000021BC1E493A3F8E493A34003F68001F201
:1019300008DFF48029E493A3F85407240CC8C333C8
:10194000C4540F4420C8834004F456800146F6DF97
:10195000E4800B0102040810204080900006E47E21
:10196000019360BCA3FF543F30E509541FFEE4938C
:10197000A360010ECF54C025E060A840B8E493A353
:10198000FAE493A3F8E493A3C8C582C8CAC583CA7E
:10199000F0A3C8C582C8CAC583CADFE9DEE780BE36
:01000A0000F5
:00000001FF
